:100000000C9455020C947D020C947D020C947D029C
:100010000C947D020C947D020C947D020C947D0264
:100020000C947D020C947D020C947D020C947D0254
:100030000C947D020C947D020C947D020C947D0244
:100040000C9440280C947D020C943D2A0C948B2A2D
:100050000C947D020C947D020C947D020C947D0224
:100060000C947D020C947D02FB15D5155C1750167F
:100070003A160917E7155C171716CC15DE15F81692
:100080003D1659174517F015121659174C17E41657
:10009000ED160017FB165C179A029E02A302A70238
:1000A000B102B602BD02C202C802CD02D202D7021C
:1000B000DE02E602EE02F402F902FF020B03130372
:1000C00018031F0326032E03485454502F312E309B
:1000D0002034303120556E617574686F72697A65AD
:1000E000640A436F6E74656E742D547970653A209E
:1000F000746578742F68746D6C0A3C68313E3430D6
:100100003120556E617574686F72697A65643C2F31
:1001100068313E0057616B652075700A004D61695A
:100120006E74656E616E63650A004C6E646B20547C
:1001300072616365722076302E38622C2028632924
:100140004C65204E6574206475204B65726D657535
:100150007220323031330A002C2047617465776198
:10016000793A20002C204E65746D61736B3A200043
:10017000495020616464726573733A2000206D56A3
:100180000A00206D562C2056696E3A2000206279B4
:100190007465732C205663633A20004672656520AF
:1001A0006D656D6F72793A20006261636B20746FC8
:1001B000203139322E3136382E312E32350A006454
:1001C0006F6E650A0052657175657374696E67209C
:1001D00049502041646472657373202E2E2E2000D6
:1001E0003C68313E323030204F4B3C2F68313E006E
:1001F0000A3C2F626F64793E0A3C2F68746D6C3E36
:100200000A003C68746D6C3E3C686561643E3C74F9
:1002100069746C653E4C6E646B20547261636572E8
:100220003C2F7469746C653E3C2F686561643E0ABE
:10023000003C626F64793E3C68313E4C6E646B20DA
:100240005472616365722076657273696F6E207691
:10025000302E38623C2F68313E0A00485454502FEB
:10026000312E3020323030204F4B0D0A436F6E74E8
:10027000656E742D547970653A20746578742F68B2
:10028000746D6C0D0A507261676D613A206E6F2D4E
:1002900063616368650D0A0D0A00414343004144F0
:1002A000445200434D440044454C45535441474556
:1002B0000044554D5000454550524F4D0047415464
:1002C0004500484953544F004C4F4144004D414371
:1002D00041004D41534B004D454D4F5259004D4546
:1002E0005355524553004D4F444545434F005041EF
:1002F00052414D00504F5254005245534554005303
:10030000455249414C4445425547005354414E449F
:1003100042590054494D4500555054494D450056E9
:10032000494E4D415800564F4C54414745005741A6
:10033000544348444F4700000108000604000145AB
:1003400000008200004000200D0A436F6E74656E4D
:10035000742D547970653A206170706C69636174B2
:10036000696F6E2F782D7777772D666F726D2D758B
:10037000726C656E636F6465640D0A0D0A00436FED
:100380006E74656E742D4C656E6774683A20000D4E
:100390000A557365722D4167656E743A204574681D
:1003A0006572536869656C642F312E360D0A41639E
:1003B000636570743A202A2F2A0D0A436F6E6E65AA
:1003C0006374696F6E3A20636C6F73650D0A000D7C
:1003D0000A0020485454502F312E310D0A486F73B3
:1003E000743A2000504F5354200020000D0A5573DA
:1003F00065722D4167656E743A2045746865725365
:100400006869656C642F312E360D0A41636365702F
:10041000743A20746578742F68746D6C0D0A436F9C
:100420006E6E656374696F6E3A20636C6F73650DF1
:100430000A0D0A0020485454502F312E310D0A481D
:100440006F73743A200047455420000000000024D8
:100450000027002A0000000000250028002B0000D3
:1004600000000023002600290004040404040404FE
:100470000402020202020203030303030301020453
:100480000810204080010204081020010204081016
:100490002000000007000201000003040600000025
:1004A0000000000000009707F92B11241FBECFEFBA
:1004B000D8E0DEBFCDBF15E0A0E0B1E0E2E7FDE5AA
:1004C00002C005900D92AE39B107D9F717E0AEE939
:1004D000B5E001C01D92A43CB107E1F714E0CAEAFF
:1004E000D4E004C02297FE010E947C2EC63AD107B8
:1004F000C9F70E944F2C0C94B72E0C940000A0E07A
:10050000B0E0E5E8F2E00C94882EEC01A880B98018
:10051000CA80DB80A114B104C104D10441F484E297
:10052000A82E89EDB82E8BE5C82E87E0D82EC601FF
:10053000B5012DE133EF41E050E00E945F2E27EA44
:1005400031E440E050E00E94F72D7B018C01C601B0
:10055000B5012DE133EF41E050E00E945F2ECA016A
:10056000B9012CEE34EF4FEF5FEF0E94F72D6E0DC7
:100570007F1D801F911F97FF04C061507040804015
:100580009048688379838A839B839B013F77C90165
:10059000CDB7DEB7EAE00C94A42E0E947F02089546
:1005A00084E291E00E947F020895A0E0B0E0809391
:1005B000240190932501A0932601B093270108956B
:1005C000FC0105900020E9F7809590958E0F9F1F04
:1005D0000895FB01DC014150504030F08D910590B1
:1005E000801919F40020B9F7881B990B0895DC01D4
:1005F00001C06D9341505040E0F70895FB01DC01CC
:100600004150504030F08D910190801919F4002034
:10061000B9F7881B990B0895EF92FF920F931F93E0
:10062000CF93DF93EC01A0E0B0E0EE24FF2487013C
:1006300009C0F901EA0FFB1F8081E80EF11C011DC2
:10064000111D1196A617B707A4F3452B69F09B015E
:10065000442737FD4095542FB701C8010E943D2E15
:10066000C901DA017C018D01D801C701807F90703A
:10067000A070B07024E0B695A795979587952A95B8
:10068000D1F78A3010F0895C01C0805DFE01E95825
:10069000FB4F80839E012F5F3F4F6E2D6F706A303E
:1006A00010F0695C01C0605DF901E958FB4F60839F
:1006B0002F5F3F4FF901E958FB4F80E280832F5FA6
:1006C0003F4FC901DF91CF911F910F91FF90EF90A4
:1006D0000895EF92FF920F931F93CF93DF93EC0156
:1006E000FA0120E030E0EE24FF2487010AC0819166
:1006F0009191A0E0B0E0E80EF91E0A1F1B1F2F5FCA
:100700003F4F261737079CF39B01442737FD409541
:10071000542FC801B7010E943D2E79018A01D801EA
:10072000C7016CE0B695A795979587956A95D1F71F
:100730008F708A3010F0895C01C0805DFE01E9583D
:10074000FB4F80839E012F5F3F4FBB27A12F902F30
:100750008F2D8F708A3010F0895C01C0805DF901A7
:10076000E958FB4F80832F5F3F4FD801C701807F3F
:100770009070A070B07044E0B695A7959795879556
:100780004A95D1F78A3010F0895C01C0805DF9018B
:10079000E958FB4F80832F5F3F4F4E2D4F704A30FB
:1007A00010F0495C01C0405DF901E958FB4F4083FE
:1007B0002F5F3F4FF901E958FB4F80E280832F5FA5
:1007C0003F4FC901DF91CF911F910F91FF90EF90A3
:1007D00008959C01DB01CA01FCE1B695A7959795A8
:1007E0008795FA95D1F78A30910514F0895C01C09C
:1007F000805DF901E958FB4F80832F5F3F4FDB019C
:10080000CA0180709070A070BF708B2F9927AA27A3
:10081000BB278A30910514F0895C01C0805DF90125
:10082000E958FB4F80832F5F3F4FDB01CA01807087
:100830009070A07FB070F4E1B695A79597958795D5
:10084000FA95D1F78A30910514F0895C01C0805D7A
:10085000F901E958FB4F80832F5F3F4FDB01CA014D
:1008600080709070AF70B070CD01AA27BB278A301E
:10087000910514F0895C01C0805DF901E958FB4FD6
:1008800080832F5F3F4FDB01CA018070907FA07093
:10089000B070FCE0B695A79597958795FA95D1F736
:1008A0008A30910514F0895C01C0805DF901E95836
:1008B000FB4F80832F5F3F4FDB01CA0180709F7029
:1008C000A070B070892F9A2FAB2FBB278A3091056B
:1008D00014F0895C01C0805DF901E958FB4F808309
:1008E0002F5F3F4FDB01CA01807F9070A070B07016
:1008F00074E0B695A795979587957A95D1F78A3044
:10090000910514F0895C01C0805DF901E958FB4F45
:1009100080832F5F3F4F4F7050704A30510514F065
:10092000495C01C0405DF901E958FB4F40832F5FEE
:100930003F4FF901E958FB4F80E280832F5F3F4F23
:10094000C9010895DC01FC01E95AFE4FE0818E2FB8
:1009500080538A3038F08151863010F080E002C038
:100960008E2F8753982F9295907FA95ABE4F11963C
:10097000EC918E2F80538A3010F4892B08958E2F9E
:100980008154863010F080E008958E2F8753892B94
:1009900008950F931F93CF93DF938C01E091A205ED
:1009A000EE2309F400C120919E05222369F4809171
:1009B0009F05882349F48091A005882329F480911C
:1009C000A105882309F4EFC040E0A0E08A2F90E061
:1009D000880F991F50E04E1708F451E0A52FA82B5F
:1009E0004F5F483099F760E0862F90E0880F991F9D
:1009F00050E04E1708F451E0652F682B4F5F4031EF
:100A000099F770E0872F90E0880F991F50E04E17FC
:100A100008F451E0752F782B4F5F483199F780E04B
:100A200090E0880F991F50E04E1708F451E0582BC2
:100A3000852F4F5F4032A1F7F801E95AFE4F8081C0
:100A4000C82FD0E08A2F90E08C239D2330E08217BE
:100A5000930729F5862F90E0218130E082239323AC
:100A600020919F0530E082179307C9F4872F90E00B
:100A7000228130E0822393232091A00530E0821769
:100A8000930769F4852F90E0238130E0822393233C
:100A90002091A10530E08217930709F484C0E0910A
:100AA000A705EE2309F47CC02091A305222369F455
:100AB0008091A405882349F48091A505882329F411
:100AC0008091A605882309F46BC0F72F40E08F2F93
:100AD00090E0880F991F50E04E1708F451E0F52F71
:100AE000F82B4F5F483099F7672F862F90E0880FDB
:100AF000991F50E04E1708F451E0652F682B4F5FA7
:100B0000403199F7872F90E0880F991F50E04E17DA
:100B100008F451E0752F782B4F5F483199F750E07A
:100B2000852F90E0880F991F50E04E1708F451E090
:100B3000A52FA82B5A2F4F5F403291F78F2F90E0AF
:100B40008C239D2330E08217930751F5862F90E088
:100B5000F801E95AFE4F218130E08223932320914E
:100B6000A40530E082179307D9F4872F90E0228103
:100B700030E0822393232091A50530E0821793076C
:100B800079F440E050E08A2F90E0238130E0822326
:100B900093232091A60530E08217930731F403C018
:100BA00040E050E002C041E050E0CA01DF91CF9147
:100BB0001F910F910895FC0150814181A82FFC01E4
:100BC00070E062507040B0E131E416C0228190E0E4
:100BD000852F880F47FD8F5F440F27FD4F5F57FD1F
:100BE00002C0582F03C0582F5B2743279F5F9830C0
:100BF00011F0220FEDCF31968E2F8A1B90E08617D1
:100C0000970724F3952F80E0242F30E0282B392BF1
:100C1000C90108952F923F924F925F926F927F92F7
:100C20008F929F92AF92BF92CF92DF92EF92FF92FC
:100C30000F931F93DF93CF93CDB7DEB728970FB6EF
:100C4000F894DEBF0FBECDBF809117048B3E09F034
:100C500055C180911804803909F050C18091190460
:100C60008B3E09F04BC180911A04803909F046C1CE
:100C700080911B048B3E09F041C180911C04803996
:100C800009F03CC187ED95E09C838B83EBEEF5E0AA
:100C9000FA83E9838FEF282E85E0382E03E1602E5A
:100CA00006E0702E17E2812E16E0912EBBE3AB2EEC
:100CB000B6E0BB2EA5E4CA2EA6E0DA2EFFE4EF2EA6
:100CC000F6E0FF2E09E516E063E676E04DE656E035
:100CD00027E736E081E896E098878F83ABE8B6E0B7
:100CE000E5E9F6E0FE83ED83E8E04E2E512CEB8142
:100CF000FC8180899189938B828BE981FA8180893B
:100D00009189938B828BF10180899189938B828B5E
:100D1000F30180899189938B828BF4018089918979
:100D2000938B828BF50180858187F6018085818791
:100D3000F70180858187F80180858187FB018085A7
:100D40008187FA0180858187F90180858187EF811C
:100D5000F8858085818718968C91189719968C93C1
:100D60001997ED81FE8180899189938B828B0894FC
:100D7000410851088B819C8102979C838B83E98178
:100D8000FA813297FA83E9838EEF9FEF280E391E9E
:100D9000680E791E880E991E0894A108B10808945F
:100DA000C108D1080894E108F108015010406150D1
:100DB00070404150504021503040EF81F8853197CC
:100DC000F887EF8311978D819E8102979E838D8393
:100DD0009FEF49169FEF590609F089CF90912104A2
:100DE00080E02091200430E0822B932B9093D80553
:100DF0008093D7059091230480E02091220430E075
:100E0000822B932B9093EC058093EB059091270414
:100E100080E02091260430E0822B932B90930006F3
:100E20008093FF059091290480E02091280430E010
:100E3000822B932B909314068093130690912B048E
:100E400080E020912A0430E0822B932B9093280697
:100E50008093270680912C0480933B0680912D047B
:100E60008093450680912E0480934F0680912F0435
:100E700080935906809130048093630680913104F9
:100E800080936D06809132048093770680913304BD
:100E9000809381068091340480938B069091360470
:100EA00080E02091350430E0822B932B90939606BE
:100EB00080939506109138040091390410923904FA
:100EC000109238048DE194E06DE10E94DB051093EF
:100ED00038040093390490933B0480933C04809140
:100EE000C0059091C10501969093C1058093C005FE
:100EF0001092A9051092A8051092770428960FB6B3
:100F0000F894DEBF0FBECDBFCF91DF911F910F913F
:100F1000FF90EF90DF90CF90BF90AF909F908F9019
:100F20007F906F905F904F903F902F90089584EC4A
:100F300095E00E9489260895AC0184EC95E067E570
:100F400071E020EF31E00E9433270895EF92FF9285
:100F50000F931F93AC0104EC15E097E5E92E91E0A7
:100F6000F92EC801B70122E032E00E943327AC011C
:100F7000C801B70121E332E00E9433271F910F918E
:100F8000FF90EF90089584EC95E067E571E040E014
:100F900050E02BE532E00E94332708958EE48093E1
:100FA0007C0062E070E080E090E00E9496288091F2
:100FB0007A00806480937A0080917A0086FDFCCF6D
:100FC0008091780090E0A0E0B0E060917900362F49
:100FD00020E0442737FD4095542F282B392B4A2BEE
:100FE0005B2B60E070E381E190E00E945F2ECA011C
:100FF000B9010895CF93DF93EC010CC06A3029F456
:101000008EE897E00E94902C04C08EE897E00E9442
:10101000B72B2196FE016491662381F7DF91CF9172
:101020000895AF92BF92CF92DF92EF92FF920F930B
:101030001F93CF93DF935C014091D3055091D4056A
:101040004115510579F0C091D505D091D605FE0125
:10105000EE0FFF1FE856FF4F659174910E94E90261
:10106000892B19F1CC24DD2447E1E42EF12CE60193
:10107000CE0DDF1DD595C795D093D605C093D50568
:10108000FE01EE0FFF1FE856FF4F05911491C801B6
:101090000E94E002AC019093D4058093D305C50172
:1010A000B8010E94E902009719F4FE01B09611C040
:1010B000181619062CF46E010894C11CD11C04C02A
:1010C0007E010894E108F108EC14FD0484F6E0E0E8
:1010D000F0E0CF01DF91CF911F910F91FF90EF9042
:1010E000DF90CF90BF90AF9008950E94C3070E94F9
:1010F000A607AC0184EC95E067E571E027E734E0F2
:101100000E942D270E949C0708950F931F93CF9351
:10111000DF938C010E94CD270E949227805D8093EF
:1011200077048091C0059091C105409734F08FE01D
:1011300090E09093C1058093C0058091C005909187
:10114000C1058A30910514F0895C01C0805D8093EF
:10115000780480E3809379048091BE05805D80935C
:101160007A0480E280937B040E94CD27AB01BC010E
:1011700085E090E00E94E903FC011016110634F5A9
:10118000C7E1D4E0DC01A958BB4F20E29881892F48
:1011900082958F708A3010F0895C01C0805D8C93DD
:1011A000892F8F708A3010F0895C01C0805D1196A4
:1011B0008C93119712962C9312972196139684E094
:1011C000CF33D80719F7E858FF4F6DC06091C005BD
:1011D0007091C105161617060CF065C0EB016B3057
:1011E000710514F0CAE0D0E0CF01BE0147ED55E033
:1011F0000E946903BE014BEE55E00E946903BE01E7
:101200004FEF55E00E946903BE0143E156E00E94A2
:101210006903BE0147E256E00E946903BE0145E949
:1012200056E00E946903BE0140E050E02BE336E047
:101230000E940C03BE0140E050E025E436E00E942D
:101240000C03BE0140E050E02FE436E00E940C03A6
:10125000BE0141E050E029E536E00E940C03BE01EA
:1012600040E050E023E636E00E940C03BE0140E07F
:1012700050E02DE636E00E940C03BE0140E050E055
:1012800027E736E00E940C03BE0140E050E021E871
:1012900036E00E940C03BE0141E050E02BE836E04E
:1012A0000E940C03FC01F093AB05E093AA05E958FA
:1012B000FB4F108287E591E00E947508012B21F415
:1012C0001092C1051092C005DF91CF911F910F912F
:1012D00008955F926F927F928F929F92AF92BF928A
:1012E000CF92DF92EF92FF920F931F93CF93DF93F2
:1012F0003C010E94CD270E949227805D8093770455
:101300008091C0059091C105409734F08FE090E046
:101310009093C1058093C0058091C0059091C1054F
:101320008A30910514F0895C01C0805D8093780457
:1013300080E3809379048091BE05805D80937A0478
:1013400080E280937B040E94CD27AB01BC0185E045
:1013500090E00E94E903EC0185E10E943429AA246F
:10136000BB24812CE4E09E2E00E010E0CC24DD24A0
:10137000760170E2572E64E170E080E090E00E9418
:10138000962885E10E9434299C01881599050CF462
:101390004C01021713070CF489016114710429F040
:1013A00084E0A816B10409F047C0E3E0293E3E07F7
:1013B00064F0FE01E958FB4FC90168EE73E00E943A
:1013C0002A2E605D6083219603C02536310584F0A6
:1013D000FE01E958FB4FC90168EE73E00E942A2E16
:1013E00064E670E00E942A2E605D6083219603C04F
:1013F0002B3031057CF0FE01E958FB4FC90164E652
:1014000070E00E942A2E6AE070E00E942A2E605D41
:1014100060832196FE01E958FB4FC9016AE070E044
:101420000E942A2E805D8083CE010196FC01E9583E
:10143000FB4F5082EC012196C901AA2797FDA09588
:10144000BA2FC80ED91EEA1EFB1E0894A11CB11C9F
:10145000F7E0AF16B10409F08ECF080D191DC801D1
:10146000AA2797FDA095BA2FC81AD90AEA0AFB0A3B
:10147000A0904301B0904401950140E050E0C701C5
:10148000B6010E94F72D20E034E140E050E00E94D8
:101490003D2E69017A01FE01E958FB4F88E2808305
:1014A000219681E1C81687E2D80680E0E80680E050
:1014B000F80680F08E0109581B4FC701B60120E1E4
:1014C00037E240E050E00E943D2E205DF80120838D
:1014D000219609C0F9EECF16F3E0DF06F0E0EF0643
:1014E000F0E0FF06B0F08E0109581B4FC701B601AE
:1014F00020E137E240E050E00E943D2E28EE33E04C
:1015000040E050E00E943D2E205DF80120832196AE
:1015100006C0F5E6CF16D104E104F104B0F08E0167
:1015200009581B4FC701B60128EE33E040E050E0F8
:101530000E943D2E24E630E040E050E00E943D2E27
:10154000205DF8012083219606C0FBE0CF16D10470
:10155000E104F104A8F08E0109581B4FC701B60140
:1015600024E630E040E050E00E943D2E2AE030E0EA
:1015700040E050E00E943D2E205DF801208321963E
:101580008E0109581B4FC701B6012AE030E040E048
:1015900050E00E943D2E605DF8016083CE0101960F
:1015A000FC01E958FB4F30E230830196FC01E95819
:1015B000FB4F2DE620830196FC01E958FB4F26E501
:1015C00020830196FC01E958FB4F29E22083DC01CE
:1015D0001196672809F47DC0FD01E958FB4F30835F
:1015E000CD010196FC01E958FB4F2DE420830196C3
:1015F000FC01E958FB4F21E620830196FC01E958E4
:10160000FB4F28E720830196FC01E958FB4F2AE3B2
:1016100020839C012F5F3F4FF1E1AF16F7E2BF0639
:1016200068F0F901E958FB4FC50160E177E20E94DB
:10163000162E605D60832F5F3F4F05C089EEA816B0
:1016400083E0B80688F0F901E958FB4FC50160E175
:1016500077E20E94162E68EE73E00E94162E605DFF
:1016600060832F5F3F4F04C0E5E6AE16B10488F0FB
:10167000F901E958FB4FC50168EE73E00E94162E90
:1016800064E670E00E94162E605D60832F5F3F4F1E
:1016900004C0FBE0AF16B10480F0F901E958FB4F3C
:1016A000C50164E670E00E94162E6AE070E00E94B8
:1016B000162E605D60832F5F3F4FF901E958FB4FA5
:1016C000C5016AE070E00E94162E805D8083D9011A
:1016D0001196A958BB4F1C9287E591E00E947508AE
:1016E000DF91CF911F910F91FF90EF90DF90CF90FE
:1016F000BF90AF909F908F907F906F905F90089574
:101700000F931F93DF93CF9300D0CDB7DEB70E9426
:101710009227805D809377048091C0059091C105E8
:10172000409734F08FE090E09093C1058093C0051E
:101730008091C0059091C1058A30910514F0895CB3
:1017400001C0805D8093780480E380937904809168
:10175000BE05805D80937A0410E210937B040E94A2
:10176000CD27AB01BC0185E090E00E94E903FC01BC
:10177000E958FB4F26E420830196FC01E958FB4F12
:1017800022E720830196FC01E958FB4F25E62083E0
:101790000196FC01E958FB4F20830196FC01E958B2
:1017A000FB4F2AE320830196FC01E958FB4F10838D
:1017B0008C010F5F1F4F8091C0079091C107009768
:1017C00011F484EC97E09E012F5F3F4F281B390BEB
:1017D00087E22031380718F020E030E038C083E09D
:1017E000293E38076CF0F801E958FB4FC90168EE53
:1017F00073E00E942A2E605D60830F5F1F4F03C05D
:10180000253631058CF0F801E958FB4FC90168EE27
:1018100073E00E942A2E64E670E00E942A2E605D2A
:1018200060830F5F1F4F03C02B30310584F0F80138
:10183000E958FB4FC90164E670E00E942A2E6AE075
:1018400070E00E942A2E605D60830F5F1F4FF801D9
:10185000E958FB4FC9016AE070E00E942A2E805DC2
:101860008083F8013196DF01A958BB4F80E28C9349
:101870003196DF01A958BB4F82E68C933196DF0188
:10188000A958BB4F89E78C933196DF01A958BB4F0C
:1018900084E78C933196DF01A958BB4F85E68C9382
:1018A000E858FB4F83E78083118287E591E00E942F
:1018B00075080F900F90CF91DF911F910F910895B0
:1018C0000F931F930E949227805D809377048091ED
:1018D000C0059091C105409734F08FE090E090935F
:1018E000C1058093C0058091C0059091C1058A30E3
:1018F000910514F0895C01C0805D8093780480E3D9
:10190000809379048091BE05805D80937A0480E2A3
:1019100080937B040E94CD27AB01BC0185E090E061
:101920000E94E9038C010E94CD27AB01BC0180918C
:10193000AE059091AF05A091B005B091B105481BDF
:10194000590B6A0B7B0BC8010E94E903FC019093C1
:10195000AB058093AA05E958FB4F108287E591E01B
:101960000E9475081F910F9108957F928F929F9208
:10197000AF92BF92CF92DF92EF92FF920F931F939D
:10198000CF93DF93EC01672B09F4A8C080E091E0CE
:10199000BE0144E050E00E94FE02009709F09EC0A4
:1019A000FC8005E010E0AA24BB2465011DC0C6012F
:1019B000B5012AE030E040E050E00E94F72D2F2DE5
:1019C000332727FD3095205330405901CC24B7FCF4
:1019D000C094DC2CA60EB71EC81ED91EFE01E00F57
:1019E000F11FF0800F5F1F4F8F2D80538A3018F446
:1019F0000F301105E1F6B801615070406C0F7D1F8A
:101A000085E091E044E050E00E94FE02009709F07A
:101A100047C0FE01E00FF11F7380A4E08A2E912CD5
:101A2000800E911EEF01EE24FF2487011BC0C80128
:101A3000B7012AE030E040E050E00E94F72D272D6A
:101A4000332727FD30952053304079010027F7FCDC
:101A50000095102FE60EF71E081F191F7B800894B3
:101A6000811C911C872D80538A3028F4219669E1CE
:101A700086169104E4F2A8019701D801C70188579E
:101A80009040A040B040895A9B41A040B04020F017
:101A900020EB34E040E050E0CA01B9010E949727F2
:101AA0000E949227892BB1F40E94882828EE33E007
:101AB00040E050E00E943D2ED601C501821B930BF1
:101AC000A40BB50B8093AE059093AF05A093B00522
:101AD000B093B105C601B5010E94A0270E94600C19
:101AE000DF91CF911F910F91FF90EF90DF90CF90FA
:101AF000BF90AF909F908F907F900895CF92DF928C
:101B0000EF92FF920F931F93CF93DF9391E0909307
:101B100077048093780460937904A9EAB6E0CAE771
:101B2000D4E0E62FF0E09F012A0F3B1F02C08D9109
:101B30008993A217B307D9F71AE7E12E14E0F12E23
:101B4000EE0EFF1ED7011C928F0105581B4FD801C6
:101B50001C92B5E0CB2ED12CCE0EDF1EF601E9583B
:101B6000FB4F8FE780836B5F87E794E00E94DB0584
:101B7000F7019083D8018C93C0E0D0E08091C2053A
:101B80009091C305892B59F08EE897E06BEE0E9487
:101B9000B72B8EE897E060E90E94B72B1AC08EE859
:101BA00097E06BEE70E040E150E00E94912D8EE8EE
:101BB00097E060E20E94882C8EE897E060E970E090
:101BC00040E150E00E94912D8EE897E060E20E9493
:101BD000882C2196C330D10589F6C7E7D4E000E010
:101BE00010E08091C2059091C305892B21F08EE809
:101BF00097E068810AC08EE897E0688140E150E094
:101C00000E943F2D8EE897E060E20E94B72B0F5FA5
:101C10001F4F2196C016D10624F78091C2059091DE
:101C2000C305892B21F48EE897E00E94902CDF9168
:101C3000CF911F910F91FF90EF90DF90CF9008957B
:101C40001092A906892B19F081E08093A9061092C1
:101C5000AA068AEA61E00E947E0D0895CF93DF9381
:101C6000C0E0D0E08CEE96E0BE010E947F27FE012E
:101C7000E95EFB4F80832196C034D10599F710921D
:101C80005704809117048D34A9F58091180481348C
:101C900089F55091190440911A0430911B04209148
:101CA0001C0490911D0480911E04552359F4442373
:101CB000A9F4332399F4222389F4992379F488230E
:101CC00069F418C05F3F51F44F3F41F43F3F31F496
:101CD0002F3F21F49F3F11F48F3F61F05093280173
:101CE0004093290130932A0120932B0190932C01DA
:101CF00080932D0180911F04813421F5809120046F
:101D0000843401F5809121048434E1F4809122042B
:101D10008235C1F43091230420912404909125044C
:101D2000809126043F3F31F42F3F21F49F3F11F46F
:101D30008F3F41F030932E0120932F01909330017B
:101D40008093310180912F04873469F580913004AC
:101D5000813449F580913104843529F5809132042C
:101D6000853409F530913304209134049091350481
:101D700080913604332339F4222369F4992359F4EA
:101D8000882349F410C03F3F31F42F3F21F49F3F97
:101D900011F48F3F41F0309332012093330190933F
:101DA000340180933501809137048035B1F48091FE
:101DB00038048F3491F480913904823571F4809124
:101DC0003A04843551F480913B0490913C0488237B
:101DD00011F4992311F09093420180913D048134D4
:101DE00009F073C080913E04833409F06EC0809185
:101DF0003F04833409F069C080914004813309F0C5
:101E000064C0409141043091420420914304909178
:101E1000440450914504852F8150803208F055C00C
:101E2000442339F4332371F4222361F4992351F4C8
:101E30004CC04F3F39F43F3F29F42F3F19F49F3FE7
:101E400009F443C040939E0530939F052093A0055D
:101E50009093A1055093A205809146048134A9F581
:101E600080914704833489F580914804833469F56F
:101E700080914904823349F540914A0430914B04E2
:101E800020914C0490914D0450914E04852F815027
:101E90008032D8F4442339F4332369F4222359F4EB
:101EA000992349F412C04F3F31F43F3F21F42F3FB3
:101EB00011F49F3F51F04093A3053093A405209364
:101EC000A5059093A6055093A70580914F048234F1
:101ED000E1F4809150048635C1F480915104893435
:101EE000A1F4809152048E3481F4209153043091F6
:101EF0005404222311F4332341F0922F80E0830F06
:101F0000911D909344018093430180915B0483353C
:101F1000E1F480915C048435C1F480915D048234E5
:101F2000A1F480915E048C3481F420915F0430919F
:101F30006004222311F4332341F0922F80E0830FB9
:101F4000911D9093480180934701809161048335EE
:101F5000E1F4809162048F34C1F48091630483348E
:101F6000A1F480916404883481F420916504309157
:101F70006604222311F4332341F0922F80E0830F73
:101F8000911D90934A0180934901809167048335A4
:101F9000E1F4809168048F34C1F480916904833442
:101FA000A1F480916A048C3481F420916B04309107
:101FB0006C04222311F4332341F0922F80E0830F2D
:101FC000911D90934C0180934B01DF91CF91089527
:101FD0005F926F927F928F929F92AF92BF92CF92B9
:101FE000DF92EF92FF920F931F93CF93DF937C01C9
:101FF0000E94C3070E94A6076C01F694FE2CEE24F3
:10200000F794E7948F2D8F708A3010F0895C01C0AF
:10201000805D80937704C701B4E096958795BA9563
:10202000E1F78870805D8093780480E38093790481
:102030008AE380937A0480E280937B048701C5E081
:10204000D0E0A0E8AA2EB12CAE0CBF1CFDE05F2EA4
:10205000EAE06E2E70E3772E6AE3862E50E2952E2C
:1020600084C0E016F1060CF057C0C8018F70907064
:10207000892B09F051C0FE01E958FB4F5082CE0177
:102080000196FC01E958FB4F60829C012F5F3F4F96
:10209000812F8F708A3010F0895C01C0805DF9015A
:1020A000E958FB4F80832F5F3F4FC801807F9070BE
:1020B00044E0959587954A95E1F78A3010F0895C60
:1020C00001C0805DF901E958FB4F8083C901019689
:1020D000FC01E958FB4F70820196FC01E958FB4F67
:1020E00080820196FC01E958FB4F9082EC01219619
:1020F000C8018F739070892B79F4C958DB4F18820F
:1021000084EC95E067E571E0A60127E734E00E94E2
:102110002D276C01C0E0D0E08CEE96E0B8010E9463
:102120007F27982F92959F70282F2F709A3018F044
:10213000892F895C02C0892F805DFE01E958FB4F21
:102140008083CE0101962A3010F0295C01C0205D09
:10215000FC01E958FB4F20830196FC01E958FB4F35
:102160009082EC0121960F5F1F4F0A151B0509F0A5
:1021700078CFC958DB4F188284EC95E067E571E0B1
:10218000A60127E734E00E942D270E949C07DF91DB
:10219000CF911F910F91FF90EF90DF90CF90BF9064
:1021A000AF909F908F907F906F905F900895CF92A7
:1021B000DF92EF92FF920F931F93CF93DF938C01E7
:1021C0007B01EA0169018CEE96E06EE370E043E585
:1021D0000E9486278CEE96E06FE370E044E50E9453
:1021E00086278CEE96E060E470E042E40E94862749
:1021F0008CEE96E061E470E048E40E9486278CEE65
:1022000096E062E470E0412F0E9486278CEE96E013
:1022100063E470E0402F0E9486278CEE96E064E431
:1022200070E043E50E9486278CEE96E065E470E05E
:1022300044E50E9486278CEE96E066E470E042E476
:102240000E9486278CEE96E067E470E04CE40E94E2
:1022500086278CEE96E068E470E04F2D0E9486277A
:102260008CEE96E069E470E04E2D0E948627209760
:1022700009F45FC01C141D040CF05BC0CC16DD0615
:1022800008F057C08CEE96E06AE470E043E50E94E7
:1022900086278CEE96E06BE470E04FE40E94862780
:1022A0008CEE96E06CE470E043E40E9486278CEEAE
:1022B00096E06DE470E048E40E9486278CEE96E09C
:1022C0006EE470E04D2F0E9486278CEE96E06FE45E
:1022D00070E04C2F0E9486278CEE96E060E570E05F
:1022E00043E50E9486278CEE96E061E570E04FE4BE
:1022F0000E9486278CEE96E062E570E043E40E943F
:1023000086278CEE96E063E570E04CE40E94862719
:102310004D2D552747FD5A958CEE96E064E570E00B
:102320000E9486278CEE96E065E570E04C2D0E94B9
:102330008627DF91CF911F910F91FF90EF90DF9053
:10234000CF9008954F925F926F927F928F929F925B
:10235000AF92BF92CF92DF92EF92FF920F931F93B3
:10236000CF93DF933C0180E091E0B30144E050E083
:102370000E94FE02009709F02FC1F3011481C5E00D
:10238000D0E08824992454011CC0C501B4012AE07E
:1023900030E040E050E00E94F72D212F332727FD49
:1023A0003095205330404901AA2497FCA094BA2CC0
:1023B000860E971EA81EB91EF301EC0FFD1F10819B
:1023C0002196812F80538A3018F4CA30D105E9F65E
:1023D000BE0161507040660D771D85E091E044E0DC
:1023E00050E00E94FE02009709F0F6C0F301EC0FE6
:1023F000FD1F53808E010C5F1F4FEF01CC24DD24A5
:1024000076011AC0C701B6012AE030E040E050E092
:102410000E94F72D252D332727FD3095205330407E
:102420006901EE24D7FCE094FE2CC60ED71EE81EF0
:10243000F91E5B800F5F1F4F852D80538A3020F47B
:10244000219605311105F4F2B80161507040660D16
:10245000771D8AE091E044E050E00E94FE02009780
:1024600009F07DC0A8014A5F5F4FF301E00FF11F43
:102470002381E8012496F301E00FF11F00E010E052
:1024800014C0C801B3E0880F991FBA95E1F7000F97
:10249000111F080F191F822F992787FD9095080F8C
:1024A000191F0053104023812196822F80538A30B8
:1024B00020F431964C175D0724F72801BE016150C6
:1024C0007040660D771D8FE091E044E050E00E947F
:1024D000FE02009719F020E030E02CC0DE011696D5
:1024E000F301EC0FFD1F6381AE014C5F5F4FF30101
:1024F000EC0FFD1F20E030E015C0C90173E0880F2C
:10250000991F7A95E1F7220F331F280F391F862F65
:10251000992787FD9095280F391F205330406381FC
:102520004F5F5F4F862F80538A3020F43196A41777
:10253000B5071CF70436110594F4201731077CF415
:102540000333110564F0293231054CF010934A0130
:102550000093490130934C0120934B0104C0442463
:10256000552420E030E0C814D904EA04FB04A0F5A7
:10257000F8E38F16F1E39F06F0E0AF06F0E0BF0648
:1025800058F181E488168AE6980680E0A80680E083
:10259000B80610F5E0E7CE16E0E3DE06E0E0EE0672
:1025A000E0E0FE06C8F0F1E9CF16F5E6DF06F0E060
:1025B000EF06F0E0FF0680F490924601809245011C
:1025C000D0924801C0924701C401B601A2010E9405
:1025D000D710C1E0D0E002C0C0E0D0E00E94C30745
:1025E0000E94A607AC01CD2B49F08FE480937704BD
:1025F0008BE680937804E2E0F0E00AC085E4809303
:10260000770482E78093780480937904E3E0F0E034
:10261000E958FB4F8AE08083118284EC95E067E5FE
:1026200071E027E734E00E942D270E949C07DF918C
:10263000CF911F910F91FF90EF90DF90CF90BF90BF
:10264000AF909F908F907F906F905F904F90089584
:10265000EF92FF920F931F937C010CEE16E0C801DE
:1026600068E370E042E40E948627C80169E370E0F5
:1026700046E50E948627C8016AE370E049E40E94AB
:102680008627C8016BE370E04EE40E9486274F2D39
:10269000552747FD5A95C8016CE370E00E948627D4
:1026A000C8016DE370E04E2D0E9486271F910F91A7
:1026B000FF90EF900895BF92CF92DF92EF92FF923A
:1026C0000F931F93CF93DF936C0180E091E0B601ED
:1026D00044E050E00E94FE02009709F049C0F60174
:1026E000B480C5E0D0E0EE24FF2487011CC0C801FF
:1026F000B7012AE030E040E050E00E94F72D2B2D9A
:10270000332727FD30952053304079010027F7FC0F
:102710000095102FE60EF71E081F191FF601EC0F8B
:10272000FD1FB08021968B2D80538A3018F4CA305B
:10273000D105E9F6D801C701815A9F40A040B040B9
:1027400080569D46A040B04098F4F0924401E0923B
:1027500043012197CC0DDD1D84E191E0BE0145E0F0
:1027600050E00E94FE02009719F4C7010E9428134E
:1027700081E090E00E946909DF91CF911F910F9154
:10278000FF90EF90DF90CF90BF9008956F927F926F
:102790008F929F92AF92BF92CF92DF92EF92FF9271
:1027A0000F931F93CF93DF936C018B01695A7E4F78
:1027B00080E091E044E050E00E94FE02009719F0B2
:1027C000C0E0D0E073C1C80104960E94A204782E34
:1027D000E8012696CE010E94A204682E80E2C81667
:1027E000D10409F473C1C80108960E94A204882E7E
:1027F000E8012A96CE010E94A204982EC114D104A9
:1028000041F086E2C816D10421F08FE2C816D10447
:1028100071F42296CE010E94A204A82EC114D10404
:1028200039F42296CE010E94A204B82E07C0AA2431
:1028300088E0C816D10409F446C0BB24772059F4B7
:10284000662049F4882039F4992029F4AA2019F443
:10285000BB2009F42BC188E1C816D10409F472C069
:1028600089E1C816D1046CF488E0C816D10461F17E
:1028700080E1C816D10409F446C0C114D10491F016
:102880000FC086E2C816D10409F49AC08FE2C816B8
:10289000D10409F495C080E2C816D10409F471C0CE
:1028A000E601BEC08CEE96E060E070E04DE40E9470
:1028B00086278CEE96E061E070E041E40E94862776
:1028C000C2E0D0E0ADC0BB248CEE96E068E070E0E2
:1028D00041E40E9486278CEE96E069E070E044E4D3
:1028E0000E9486278CEE96E06AE070E044E40E9445
:1028F00086278CEE96E06BE070E042E50E9486272A
:10290000CCE0D0E08DC08CEE96E060E170E04DE46C
:102910000E9486278CEE96E061E170E041E40E941F
:1029200086278CEE96E062E170E043E50E94862700
:102930008CEE96E063E170E04BE40E948627C4E1F0
:10294000D0E06EC08CEE96E068E170E047E40E9453
:1029500086278CEE96E069E170E041E40E948627CC
:102960008CEE96E06AE170E044E50E9486278CEEEA
:1029700096E06BE170E045E40E948627CCE1D0E070
:102980004FC08CEE96E060E270E040E50E94862742
:102990008CEE96E061E270E04FE40E9486278CEEB8
:1029A00096E062E270E042E50E9486278CEE96E0B7
:1029B00063E270E044E50E948627C4E2D0E030C0C4
:1029C00086010F5F1F4F8CEE96E0B60141E40E9436
:1029D000862778010894E11CF11C8CEE96E0B80182
:1029E00043E40E94862787010F5F1F4F8CEE96E01D
:1029F000B70143E40E948627B8016F5F7F4F86E2EC
:102A0000C816D10431F4EB018CEE96E0B80141E335
:102A100005C0EB018CEE96E0B80142E30E948627E8
:102A20008E010F5F1F4F8CEE96E0BE01472D0E9476
:102A30008627E80121968CEE96E0B801462D0E948B
:102A4000862780E2C816D10489F18E010F5F1F4FDF
:102A50008CEE96E0BE01482D0E948627E801219663
:102A60008CEE96E0B801492D0E948627C114D1044E
:102A700041F086E2C816D10421F08FE2C816D104D5
:102A8000A9F48E010F5F1F4F8CEE96E0BE014A2D18
:102A90000E948627CD2811F0E80108C0E8012196A0
:102AA0008CEE96E0B8014B2D0E948627CE01DF9177
:102AB000CF911F910F91FF90EF90DF90CF90BF903B
:102AC000AF909F908F907F906F9008958824992465
:102AD000AA24B3CEAF92BF92DF92EF92FF920F93F0
:102AE0001F93CF93DF93C091C505D091C605BE015A
:102AF000695A7E4FFB019E01AE01405C5F4F0AC0E8
:102B00009081892F81568A3110F4905290832F5FE3
:102B10003F4F31962417350720F482E0213C3807D7
:102B200078F38AE191E044E050E00E94FE020097D1
:102B300081F00E94C307AC019093C6058093C50540
:102B400084EC95E067E571E020EE31E00E943327E8
:102B5000ABC1BE01655A7E4F8FE191E042E050E08B
:102B60000E94FE02009729F487E591E00E94750813
:102B70009BC1CE01845A9E4F0E941108FC01B09760
:102B8000E831F10508F095C1EC5CFF4FEE0FFF1F37
:102B90000590F491E02D09946091C5057091C605EA
:102BA000675F7F4F80E090E023C06091C505709122
:102BB000C605675F7F4F88E090E01AC06091C50549
:102BC0007091C605675F7F4F80E190E011C0609112
:102BD000C5057091C605675F7F4F88E190E008C02A
:102BE0006091C5057091C605675F7F4F80E290E0F8
:102BF0000E94C61361C16091C5057091C605FB01B5
:102C0000E95AFE4F8085813329F4675F7F4F86E262
:102C100090E0EECF823309F04FC1675F7F4F8FE2C4
:102C200090E0E6CF109256011092550145C1C09137
:102C3000C505D091C605BE01605A7E4F80E091E087
:102C400044E050E00E94FE02009709F032C1C95AE8
:102C5000DE4F6D85603319F480E090E004C061338D
:102C600021F481E090E00E94200E81E090E00E943B
:102C700085081AC181E090E002C080E090E00E94E7
:102C800085089093C6058093C5050E9488286093A7
:102C9000BA057093BB058093BC059093BD058BC0AE
:102CA00084E190E0A0E0B0E08093B6059093B70592
:102CB000A093B805B093B905C091C505D091C605DC
:102CC000BE016B597E4F80E091E044E050E00E94ED
:102CD000FE02009709F067C01092B6051092B70582
:102CE0001092B8051092B905FE01E95AFE4FD2883C
:102CF000C3E1D0E0EE24FF2487015F011FC0C801BB
:102D0000B7012AE030E040E050E00E94F72D2D2D81
:102D100030E02053304079010027F7FC0095102F58
:102D2000E60EF71E081F191FC731D10511F4DD2467
:102D300005C0F501EC0FFD1FD08021968D2D80532D
:102D40008A3018F4C831D105D0F2E092B605F0927D
:102D5000B7050093B8051093B9058091B605909119
:102D6000B705A091B805B091B9054E97A109B10971
:102D700083569145A140B040B0F40E94CD272091E8
:102D8000B6053091B7054091B8055091B905260FA9
:102D9000371F481F591F2093B2053093B305409346
:102DA000B4055093B50582E090E09093BF05809301
:102DB000BE050E9488286093B6057093B70580937E
:102DC000B8059093B90578C08091C5059091C60566
:102DD000805A9E4F61E070E008C08091C5059091D7
:102DE000C605805A9E4F60E070E00E94B50C5CC042
:102DF0000E94800B59C080E090E00E94690954C095
:102E00008091C5059091C6058E599E4F0E945B1317
:102E10004BC0C091C505D091C605BE016E597E4F0D
:102E200080E091E044E050E00E94FE02009739F516
:102E3000FE01E95AFE4F6785FE01E959FE4F40E168
:102E400050E020E030E011C0C901A3E0880F991FD5
:102E5000AA95E1F7220F331F280F391F260F311DC6
:102E60002053304061914F5F5F4F862F80538A30EF
:102E700018F44231510541F72031310510F020E0BE
:102E800030E0C9010E94E80F0FC086E090E0909307
:102E9000BF058093BE050DC08091C5059091C60504
:102EA0008D599E4F0E94A2119093C6058093C5052F
:102EB00003C020E030E002C021E030E0C901DF9132
:102EC000CF911F910F91FF90EF90DF90BF90AF9047
:102ED0000895EF92FF920F931F93CF93DF9304E037
:102EE00010E0B3E0EB2EF12CC7E0D0E022C28091DD
:102EF000BE059091BF058330910509F4A9C08430C7
:102F0000910534F4009781F0029709F0F0C079C080
:102F10008530910509F4CCC0853091050CF4B4C01E
:102F2000069709F0E4C042C084EC95E060EC72E0E2
:102F300047E551E00E948A26AC0184EC95E067E504
:102F400071E00E948F269093C6058093C505892B5A
:102F500009F4CDC08AE190E00E94C904892B09F4EC
:102F6000C6C00E946A159093D0058093CF05892B27
:102F700009F0BDC08091BE059091BF05892B09F075
:102F8000B6C084EC95E067E571E040E050E028ECE5
:102F900030E00E9433279093C6058093C50581E0F9
:102FA00090E09093D0058093CF05A1C00E9488281F
:102FB0006093BA057093BB058093BC059093BD05E3
:102FC0002091B6053091B7054091B8055091B905EB
:102FD000621B730B840B950B673971058105910595
:102FE00008F485C081E090E00E9485089093C605B2
:102FF0008093C50581E090E09093D0058093CF0544
:1030000072C00E9488282091B6053091B705409182
:10301000B8055091B905621B730B840B950B6A3F81
:1030200071058105910508F462C081E090E00E947D
:1030300085089093C6058093C50581E090E0909344
:10304000D0058093CF05F092BF05E092BE054FC03A
:103050000E9488282091B6053091B7054091B805A7
:103060005091B905621B730B840B950B645F714023
:1030700080409040E0F11093BF050093BE0580E0D2
:1030800090E00E94200E33C00E94CD272091B2050F
:103090003091B3054091B4055091B5052617370717
:1030A0004807590720F581E090E00E94200E1BC0E0
:1030B0000E9488282091B6053091B7054091B80547
:1030C0005091B905621B730B840B950B20914D0138
:1030D00030914E0140914F0150915001621773079A
:1030E0008407950720F01092BF051092BE050E943C
:1030F0008828209151013091520140915301509103
:103100005401621B730B840B950B61537547804010
:10311000904030F18091BE059091BF05069701F176
:1031200080EA60E00E947E0D1092A9051092A80529
:103130000E94882820E335E740E050E00E943D2EC1
:10314000CA01B90120E335E740E050E00E94F72DC5
:1031500060935101709352018093530190935401F5
:103160008091CF059091D0050197E9F44091C50574
:103170005091C60584EC95E067E571E00E94282730
:10318000E7E5F1E080E090E002C01192019622E0D4
:10319000803C9207D0F39093D2058093D105109292
:1031A000D0051092CF0582E00E94E9299093D205C4
:1031B0008093D1054091CB055091CC056091CD0510
:1031C0007091CE050097D9F441155105610571053F
:1031D00059F40E9488286093CB057093CC058093A6
:1031E000CD059093CE059EC00E9488286093C705A8
:1031F0007093C8058093C9059093CA0593C0411583
:1032000051056105710509F44EC08091C705909183
:10321000C805A091C905B091CA050097A105B105DF
:1032200009F441C08E5E9240A040B040841B950BD3
:10323000A60BB70B835E9440A040B040A0F560E0C1
:1032400070E08091AC059091AD05892B11F461E09F
:1032500070E07093AD056093AC0589E00E949529FC
:103260008091AC059091AD052091C2053091C305C8
:10327000019759F4232B21F48DE191E00E94FA0784
:10328000D093BF05C093BE050EC0232B21F484E16B
:1032900091E00E94FA0781E090E00E94200E1092D7
:1032A000BF051092BE051092C7051092C805109276
:1032B000C9051092CA051092CB051092CC05109248
:1032C000CD051092CE052EC06091A8057091A9057C
:1032D000695E7B4F8EE897E041E050E00E94D32D7D
:1032E000019749F48091A8059091A90501969093C2
:1032F000A9058093A8058091A8059091A9058497B8
:1033000031F480913A048F3711F40E940A068091BB
:10331000A8059091A9058036910524F01092A90581
:103320001092A8058EE897E00E944D2B18161906FA
:103330005CF28091550190915601892B09F0D7CD0F
:10334000DF91CF911F910F91FF90EF9008950F9310
:103350001F93CF93DF938C01C0E0D0E0F801EC0F16
:10336000FD1F8EE897E060814AE050E00E943F2D0B
:10337000C330D10531F08EE897E062E271E00E943F
:10338000A42D2196C430D10549F7DF91CF911F912B
:103390000F9108954F925F926F927F928F929F92BA
:1033A000AF92BF92CF92DF92EF92FF920F931F9353
:1033B000DF93CF9300D0CDB7DEB782E060E00E940C
:1033C000562989E061E00E94562982E00E94E9299D
:1033D000019711F40E942E0E85E10E94342910E01D
:1033E000662477246AE070E080E090E00E949628EE
:1033F00085E10E943429680E791E1F5F153091F710
:10340000409043015090440181EE681685E07806B3
:1034100034F081E090E09093C3058093C2058EE87C
:1034200097E040E855E260E070E00E94C62A8EE82E
:1034300097E00E94F72B8823D1F38AE291E00E9463
:10344000FA0784EC95E00E947C2784EC95E068E222
:1034500071E00E94782780912E01882309F065C0D1
:1034600080912F01882309F060C08091300188236A
:1034700009F05BC080913101882309F056C080912A
:10348000C2059091C305892B21F485EC91E00E943F
:10349000FA0700D086E391E0EDB7FEB7928381830F
:1034A00084EC95E067E571E040EC52E028E231E021
:1034B00000E510E0BEE2EB2EB1E0FB2EAEE3CA2E3B
:1034C000A1E0DA2EF2E3AF2EF1E0BF2EEAE38E2E7A
:1034D000E1E09E2E0E9494260F900F902091C2054D
:1034E0003091C305882339F0232BF9F48FEB91E059
:1034F0000E94FA071AC0232B21F489EA91E00E9466
:10350000FA0730EC30932E0128EA20932F0191E046
:103510009093300189E180933101309332012093FF
:10352000330190933401909335012091420184EC52
:1035300095E068E271E04EE251E030E00E94392708
:1035400084EC95E062E371E00E9424278BE991E02E
:103550000E94FA078091C0079091C107009711F46B
:1035600084EC97E0BE016F5F7F4F681B790B8EE89C
:1035700097E04AE050E00E94912D8DE891E00E9492
:10358000FA070E94CE07AB01BC018EE897E02AE063
:1035900030E00E94512D82E891E00E94FA07B301C9
:1035A000882777FD8095982F920140E050E00E9497
:1035B000F72D20E034E140E050E00E943D2E8EE8FF
:1035C00097E0BA01A9012AE030E00E94302D8DE792
:1035D00091E00E94FA078091C2059091C305892B62
:1035E000E1F480E791E00E94FA078EE291E00E9408
:1035F000A71984E691E00E94FA078EE391E00E9409
:10360000A71988E591E00E94FA0782E391E00E9401
:10361000A7198EE897E00E94902C1092AB051092AB
:10362000AA051092A9051092A80581E090E00E94D9
:10363000200E1092BF051092BE0581E090E090939D
:103640005601809355010F900F90CF91DF911F91FC
:103650000F91FF90EF90DF90CF90BF90AF909F9031
:103660008F907F906F905F904F900895EF92FF92B0
:103670000F931F938091B706853011F5E090BC063B
:10368000F090BD060091BE061091BF068091B8066D
:103690009091B906A091BA06B091BB06E80EF91E4A
:1036A0000A1F1B1F0E948828AA2797FDA095BA2FE2
:1036B0008E159F05A007B10718F086E08093B70626
:1036C0008091B7061F910F91FF90EF90089585E0CC
:1036D0008093B7060E948828AA2797FDA095BA2F45
:1036E0008093B8069093B906A093BA06B093BB0630
:1036F0000E94E41E82E00895FF920F931F93CF93E0
:10370000DF938C01F62E1092C0061092C1068091B4
:10371000C2068F5F8093C20680E991E0D801FC0168
:103720001D923197E9F76091C20670E0706E40918A
:10373000B2075091B307C80124E430E00E94072289
:10374000D80116962091C3063091C406C901FC0128
:1037500086E001900D928150E1F7C8016FEF70E0B3
:1037600046E050E00E94F70282E8D80151968C931F
:10377000519781E157968C938FEF9FEFAFEFBFEF9B
:10378000F801868F978FA0A3B1A383E485A312A22B
:1037900084E483A3BA9681E0D8019A968C938183BE
:1037A00086E0828313828091B1069091B206A09147
:1037B000B306B091B40684839583A683B7838091C2
:1037C000B5069091B60691878087D801DA961D924A
:1037D0001D921D921C92DD977C962091C30630911C
:1037E000C406C901DC0186E00D9001928150E1F729
:1037F000D801AA5EBE4F93E6FD01919382E811962F
:103800008C93DF01119683E58183FD01319611963A
:103810009C93DF01119685E38183FD01319691E050
:1038200011969C93DF011196F1829D012F5F3F4F0E
:103830008DE311968C93F901319687E0D9011196A9
:103840008C939183EF0122964091C3065091C40658
:1038500020E030E0FE01E20FF31FDA01A20FB31FF8
:103860008C9180832F5F3F4F2630310599F78CE094
:103870008E838AE08F83289620E030E0FE01E20FFD
:10388000F31FD901A958BA4F8C9180832F5F3F4F06
:103890002A30310599F72A96D093C606C093C506FB
:1038A0002A97B3E0FB1609F042C082E38A8794E0CE
:1038B0009B87E091B207F091B30780818C87E091FC
:1038C000B207F091B30781818D87E091B207F09143
:1038D000B30782818E87E091B207F091B3078381AD
:1038E0008F8786E3888B998B6296D093C606C093A8
:1038F000C5066297E091B407F091B50780818A8B85
:10390000E091B407F091B50781818B8BE091B4070A
:10391000F091B50782818C8BE091B407F091B507E7
:1039200083818D8B6696D093C606C093C506A09101
:10393000C506B091C606FD0187E3819393E0119619
:103940009C93DF01119681E081839D012F5F3F4FA2
:1039500011969C93F901319686E0D90111968C93CA
:103960008FEF81833296F093C606E093C506E01B85
:10397000F10BBA97C801BF010E946523DF91CF9177
:103980001F910F91FF90089563E070E00E947C1BEF
:1039900083E08093B7060895DF92EF92FF920F9332
:1039A0001F93CF93DF938C017B01E091B207F091DD
:1039B000B307EC018AAD9BADACADBDAD8083918307
:1039C000A283B383F801E65EFE4FE00EF11EDF0135
:1039D0001196D180ED01219680818630C1F087302B
:1039E00030F4813051F0833009F057C00BC083337D
:1039F00099F0863309F051C042C0E091B807F091C8
:103A0000B90741C0E091B607F091B7073CC0E0911B
:103A1000B007F091B10737C011966C9170E080E06B
:103A200090E0982F872F762F66272981620F711DCE
:103A3000811D911D982F872F762F66272A81620F6F
:103A4000711D811D911D982F872F762F66272B8141
:103A5000620F711D811D911D982F872F762F66276C
:103A600028EE33E040E050E00E94F72D6093BC0662
:103A70007093BD068093BE069093BF060EC0E09182
:103A8000B407F091B50711968D919D910D90BC9161
:103A9000A02D80839183A283B383FE01ED0DF11DE0
:103AA000EE15FF0508F493CFC8010E94C41C81E005
:103AB000DF91CF911F910F91FF90EF90DF900895CC
:103AC000FC0166347105A0F183A1833489F5DF011F
:103AD0009A9682A5823061F514962D913D914D9173
:103AE0005C9117978091B1069091B206A091B306B0
:103AF000B091B406281739074A075B07C9F4E65E98
:103B0000FE4F8081EA51F140853391F4E45EFE4F2F
:103B10008081EC51F140823019F0853049F404C0C5
:103B2000CF010E94CC1C0895CF010E94671B08950D
:103B300080E00895CF92DF92EF92FF920F931F9350
:103B4000CF93DF93EC017093C4066093C306509348
:103B5000B3074093B2073093B9072093B807109387
:103B6000B7070093B607F092B507E092B407D0927A
:103B7000B107C092B00780E090E00E9434290E9413
:103B8000D5020E94D002AA2797FDA095BA2F8F5D7B
:103B90009C4BAA49BF4F8093B1069093B206A09365
:103BA000B306B093B4061092B6061092B50680E044
:103BB00090E0E091B207F091B307E80FF91F10828F
:103BC000E091B807F091B907E80FF91F1082E09172
:103BD000B607F091B707E80FF91F1082E091B4071C
:103BE000F091B507E80FF91F1082E091B007F0914E
:103BF000B107E80FF91F1082019684309105C9F6CC
:103C0000E091C306F091C406858182958F708F5B29
:103C100080937F0585818F708F5B809380050E94E4
:103C2000ED1ECE0161E070E00E947C1B81E080937C
:103C3000B706DF91CF911F910F91FF90EF90DF902A
:103C4000CF9008958AE061E00E9456298AE061E001
:103C50000E9495298BE061E00E9456298DE061E089
:103C60000E9456298CE060E00E9456298BE061E0BA
:103C70000E9495298BE060E00E9495298DE060E02C
:103C80000E94952981E58CBD8DB581608DBD08951B
:103C90000F931F93CF93DF938C01EB01F8948091E6
:103CA000820560E00E9495298AE78EBD0DB407FE6B
:103CB000FDCF08C088818EBD0DB407FEFDCF2196D3
:103CC0000150104001151105A9F78091820561E0AE
:103CD0000E9495297894DF91CF911F910F910895BB
:103CE0000F931F93CF93DF93EC018B01F894809196
:103CF000820560E00E9495298AE38EBD0DB407FE1F
:103D0000FDCF09C01EBC0DB407FEFDCF8EB5F80176
:103D100081938F0121972097A9F78091820561E017
:103D20000E9495297894DF91CF911F910F9108956A
:103D3000FF920F931F93082F162FF42EF894809163
:103D4000820560E00E9495291F71102B1EBD0DB4E5
:103D500007FEFDCFFEBC0DB407FEFDCF80918205AE
:103D600061E00E94952978941F910F91FF9008952A
:103D70001F93182F282F30E0207630708091C706CF
:103D800090E02817390781F080EA6FE143E00E9454
:103D9000981E412F40764093C7064295469547703E
:103DA00080E86FE10E94981E1F9108950F931F9362
:103DB000182F062F0E94B81E80E4612F402F0E940A
:103DC000981E1F910F9108956091CA066E7F6093AF
:103DD000CA0688E30E94D61E08956091CA066160F3
:103DE0006093CA0688E30E94D61E0895682F677004
:103DF00085E70E94D61E08950F931F93182F072F53
:103E00000E94D61E812F8F5F602F0E94D61E1F91A9
:103E10000F9108950F931F93182F062FF8948091F8
:103E2000820560E00E949529802F8F71812B8EBDC5
:103E30000DB407FEFDCF1EBC0DB407FEFDCF07FF7E
:103E400004C01EBC0DB407FEFDCF1EB580918205D7
:103E500061E00E9495297894812F1F910F91089518
:103E60001F93182F0E94B81E80E0612F0E940A1F26
:103E70001F910895AF92BF92CF92DF92EF92FF927F
:103E80000F931F93DF93CF9300D0CDB7DEB76C01B4
:103E90005B0189E30E94301F882319F400E010E0E1
:103EA00051C06091C8067091C90680E00E94FC1E56
:103EB00082E090E08E010F5F1F4FB8010E94701EDC
:103EC00089819A819093C9068093C80682E090E028
:103ED000B8010E94701EE980FA8082E090E0B8018B
:103EE0000E94701E898187FD03C000E010E00DC0B4
:103EF000C70104978601015010408017910708F40C
:103F00008C01C801B5010E94701E6091C8067091B5
:103F1000C9068CE00E94FC1E6091C8067091C9061B
:103F20006150704089E16F3F780720F08CE06EEFC0
:103F300079E101C08CE00E94FC1E80E86EE140E463
:103F40000E94981EC8010F900F90CF91DF911F9192
:103F50000F91FF90EF90DF90CF90BF90AF900895BA
:103F60000F931F93CF93DF93EC018B010FC08CE174
:103F70000E94301F81FF0AC080E86FE140E80E9484
:103F8000981E80EA6FE140E80E94981E80E06FE191
:103F90000E940A1F83FDEBCF82E06FEF79E10E9460
:103FA000FC1EBE016150764E86E00E94FC1E8AE730
:103FB00060E040E00E94981ECE01B8010E94481EB9
:103FC00080E86FE148E00E94981EDF91CF911F9139
:103FD0000F9108950F931F93982F162F072F84ED9D
:103FE000692F0E94D61E86ED612F0E94D61E87ED96
:103FF000602F0E94D61E04C08FE090E00E94EF2840
:104000008AEE0E94301F80FDF7CF1F910F91089517
:104010000F931F938C01862F6093820561E00E94AD
:1040200056298091820561E00E94952978948FEF4E
:1040300060E04FEF0E94981E62E370E080E090E045
:104040000E9496281092C9061092C80688E060E087
:1040500070E00E94FC1E8CE060E070E00E94FC1E9C
:104060008AE06EEF79E10E94FC1E84E06FEF79E157
:104070000E94FC1E86E06FEF7FE10E94FC1E81EB38
:104080008093CA0688E361EB0E94D61E88E26FE344
:1040900070E30E94FC1E80E369EF77EF0E94FC1E34
:1040A00080EC6DE00E94D61E81EC60E00E94D61E7E
:1040B00080E862EC42E30E94981E86EC62E17CE0BC
:1040C0000E94FC1E84EC62E10E94D61E8AEC6CED1C
:1040D00075E00E94FC1E84EEF80160810E94D61EED
:1040E00085EEF80161810E94D61E82EEF8016281A0
:1040F0000E94D61E83EEF80163810E94D61E80EED8
:10410000F80164810E94D61E81EEF80165810E944B
:10411000D61E80E160E071E00E94EA1F8FE10E94FC
:10412000B81E80E86BE140EC0E94981E80E86FE1C9
:1041300044E00E94981E1F910F910895682F84ED0E
:104140000E94D61E82ED61E00E94D61E8FE090E0B4
:104150000E94EF288AEE0E94301F80FDFBCF82ED87
:1041600060E00E94D61E89ED0E94301F90E0089505
:1041700081E10E949E2020E0892B09F021E0822F1E
:104180000895CF92DF92EF92FF920F931F93CF93F8
:10419000DF936C01413081F4685070407B0100E096
:1041A00010E0685F7F4F21E130E040E050E0E20E38
:1041B000F31E041F151F15C0423021F0EE24FF240A
:1041C00087010FC0685070407B0100E010E0685F1D
:1041D0007F4F86E090E0A0E0B0E0E80EF91E0A1FF5
:1041E0001B1FF601EB0116C0808190E0A0E0B0E05B
:1041F000BA2FA92F982F8827218130E040E050E086
:10420000822B932BA42BB52BE80EF91E0A1F1B1F24
:1042100032962297C230D10538F7FB01EE7FEC0DC4
:10422000FD1D60FF15C0808190E0A0E0B0E0BA2FD6
:10423000A92F982F882708C02FEF3FEF40E050E0CC
:10424000E222F32204231523E80EF91E0A1F1B1F86
:10425000C801AA27BB270097A105B10569F79701F7
:1042600020953095C901DF91CF911F910F91FF905B
:10427000EF90DF90CF900895CF93DF93EC015093B0
:10428000D1064093870520E030E0F901E851F94F6D
:10429000DB01A20FB31F8C9180832F5F3F4F24302F
:1042A000310599F720E030E0F901E654F84FDE01DE
:1042B000A20FB31F8C9180832F5F3F4F26303105B3
:1042C00099F7DF91CF910895FC0169327105B0F043
:1042D0008485883099F48585863081F4DF0196964F
:1042E000E8EEF6E09C918081981741F411963196A2
:1042F00086E0EC3EF807B1F781E0089580E008958C
:10430000FC016A327105D0F084858830B9F4858566
:104310008823A1F48685853489F4DF01E8EEF6E090
:104320005E969C915E978081981741F41196319624
:1043300086E0EC3EF807A1F781E0089580E008955B
:104340000F931F938C01FC01108E118E80E4848BDF
:10435000158A868BC8010E9664E170E040E00E94E9
:10436000C120F801908F818F1F910F910895AC01AA
:10437000FC01A8EEB6E0828D868F8D91828F3196FA
:1043800086E0AC3EB807B9F7CA010E94A0210895A3
:10439000FC01B99694E08081680F711D848164836B
:1043A000442311F0808301C01082915031979923EA
:1043B00019F0672F7727EFCF08950F931F938C0184
:1043C000FC0194A182A184A392A395A183A185A3BA
:1043D00093A3C8010E94C821F80112AA13AA80E57C
:1043E00086A71F910F9108956A5C7F4FDC01A60F8D
:1043F000B71F6653704003C08D936F5F7F4FFA0104
:104400004F5F5F4F84918823B9F7CB010895FF92E6
:104410000F931F93CF93DF93EC01F62E072FBA0172
:10442000122F932FAE019E01A0E0B0E0FD01E252F9
:10443000F94F8081F9018083FD01E654F84F8081B6
:10444000F901868311962F5F3F4FA630B10571F7B2
:1044500088E08C871D86DE01EFE3F3E084911E96F1
:104460008C931E973196119683E0E834F807B1F7E4
:10447000188A81E18F8BA0E0B0E0FB01EA0FFB1FFF
:104480008081FA01868FFD01E851F94F8081FA01A0
:10449000828F11964F5F5F4FA430B10571F79CA3D7
:1044A0001DA30AA3FBA21EA218A619A6DF91CF91F5
:1044B0001F910F91FF900895AC0181E080938305D7
:1044C00020E030E0F901E652F94FDA01A20FB31F04
:1044D0008C9180832F5F3F4F2430310599F70895E9
:1044E000CF93DF93EB01BA01DA010D900020E9F7D9
:1044F0001197A41BB50BE696AC014C0F5D1FE69718
:104500009D0108C0FB018191BF01FA018193AF01B8
:104510002150304021153105A9F79E012A0F3B1F7C
:10452000C901DF91CF910895FF920F931F93CF930D
:10453000DF93EC01F62E142F022FAC01DC0120E0FA
:1045400030E0F901E252F94F80818C93F901E65491
:10455000F84F808116968C9316972F5F3F4F1196D8
:104560002630310571F788E08C871D86DE01EFE388
:10457000F3E084911E968C931E973196119683E0FA
:10458000E834F807B1F78CE2898B86E08F8B20E066
:1045900030E0F901EC51F94F8081FA01868FF90181
:1045A000E851F94F8081FA01828F2F5F3F4F4F5FB3
:1045B0005F4F2430310569F7CE010E94A0211CA372
:1045C0000DA38BE08AA3FBA2FE01B69680E01192B8
:1045D0008F5F8830E1F78091880588A78D5F809391
:1045E000880580E68EA782E08FA794E098AB19AA91
:1045F0001AAA1BAA1CAA1DAA8EAB9FAB88AF86E283
:1046000089AFCE014A9660E270E042E00E94C1208C
:104610009AAB8BAB8AE390E0BE010E94B01FDF91A2
:10462000CF911F910F91FF900895CF93DF93EC01ED
:10463000AC012AEB37E0FC01D9019FEF90838D910B
:104640008683319687E0A03CB807C1F788E08C8765
:1046500086E08D87DE01E7E3F3E084911E968C937C
:104660001E973196119683E0EF33F807B1F7F90101
:1046700081919F01FA01868B10A24F5F5F4FF7E097
:10468000203C3F07A1F7DE015C9620E030E0FB0113
:10469000E20FF31F80811A968C931A97F901E85163
:1046A000F94F80818D932F5F3F4F2430310579F78B
:1046B000809183058860809383058AE290E0BE0143
:1046C0000E94B01FDF91CF910895DF92EF92FF9289
:1046D0000F931F938C017B018CE190E0E80EF91E93
:1046E000F801F08A84EE9FEFE80EF91EDE2C9CE1C3
:1046F000D90ED18AC8010E94A021E8E0F0E0EE0EB8
:10470000FF1EF801F6A2FCEEDF0EF801D7A288E04A
:1047100090E0E80EF91EC8014A96B70141E00E94F8
:10472000C120F80190A781A7C7014A96B8010E944D
:10473000B01F1F910F91FF90EF90DF900895EF92BF
:10474000FF920F931F938C017B01CB018896F80198
:10475000908B818BC8010E94A021F80112AA13AA94
:104760008CE190E0E80EF91EC8014A96B70142E0DC
:104770000E94C120F80192AB83ABC7014A96B801F1
:104780000E94B01F1F910F91FF90EF900895CF935B
:10479000DF93EC01FC01AAEBB7E0868180838D9169
:1047A0008683319687E0A03CB807B9F7842F8061F3
:1047B0008FA7443029F06115710511F461E070E0B4
:1047C000CE0141E00E94DD21188A88E2898BCE016A
:1047D0000E94B72184E088AB19AACE014A966CE109
:1047E00070E042E00E94C1209AAB8BAB86E390E080
:1047F000BE010E94B01FDF91CF910895EF92FF920A
:104800000F931F938C017B016091D2067091D306A8
:1048100040E00E94C72389E1F80187A7C801B701DA
:104820000E949F231F910F91FF90EF900895CF93C7
:10483000DF93EC01FC01AAEBB7E0868180838D91C8
:104840008683319687E0A03CB807B9F7188A8CE2D6
:10485000898BCE010E94B72182E18FA7CE0161E052
:1048600070E040E00E94DD211EA21FA28091880519
:1048700088A719A68D5F8093880582E08EAB84E0BF
:104880008FAB95E098AF19AE80E68EA798AB88E71E
:1048900089ABCE014A9660E270E042E00E94C120FE
:1048A0009AAB8BAB8AE390E0BE010E94B01FDF9110
:1048B000CF9108950F931F93CF93DF93EC018B015A
:1048C000FC01AAEBB7E0868180838D9186833196C7
:1048D00087E0A03CB807B9F7CE010E94B7211AA221
:1048E0008CA1883F18F08DA18F5F8DA38CA1885F6C
:1048F0008CA3C801BE010E94B01FDF91CF911F9110
:104900000F910895CF93DF93AC01EC012AEB37E0D0
:10491000FC01D901868180838D918683319687E061
:10492000A03CB807B9F7FA01148A82E0858B8E891A
:1049300088A3F90181919F018E8B2196F7E0203C9D
:104940003F07A9F7FA017C96A8EEB6E0808182873E
:104950008D91819386E0AC3EB807C1F78AE290E082
:10496000BA010E94B01FDF91CF910895EF92FF929C
:104970000F931F93CF93DF93EC017B0161157105BA
:1049800009F040C08091830580FD04C080918305BB
:1049900082FF0FC08091840590918505892B49F491
:1049A0000E94B820882329F0CE016AED76E00E94AB
:1049B0001523809184059091850501969093850536
:1049C000809384058091CB06813009F08FC180915E
:1049D000830581FF8BC182E08093CB0680918605A1
:1049E0008F5F809386058F716091CC066295660F0C
:1049F000607E682BCE014091CD062091CE060E94AC
:104A0000942274C10E946421882341F18D898130F0
:104A100019F4CE010E9482248091830583FF66C130
:104A20008D89823009F062C1EAEDF6E0DE015C9624
:104A30009C915C978081981709F058C11196319626
:104A400086E0EE3DF80799F7EEEDF6E08E8981936A
:104A5000219696E0E43EF907C9F752C1CE01B701AD
:104A60000E948021882309F441C19F89913149F432
:104A70008AA18823C9F48BA18533B1F46AE270E07E
:104A800037C1913089F48AA1883071F4E091D80659
:104A9000F091D906309719F0CE014A960995CE01CA
:104AA000B7010E945A2422C186E3E816F10418F4E3
:104AB000963009F01BC19CA19B3009F0C9C0D0936E
:104AC000D006C093CF06DE01E4EEF6E05A969C9144
:104AD0005A978081981709F009C11196319696E08E
:104AE000E83EF90799F710C1E091D406F091D50698
:104AF000309709F4A3C08DA182958695877063E0F5
:104B000040E050E020E030E0099598C0988980E0CE
:104B10002989022F10E0082B192B8EA582958F7002
:104B2000482F50E0CA01880F991F880F991F081B52
:104B3000190B0451104017FF02C000E010E0B8014B
:104B40008091CB06823089F531FF20C034FF1EC032
:104B5000CE0160E070E040E00E94C72388E18FA7AB
:104B6000E091D606F091D706309719F460E070E036
:104B700006C08BA18295869587700995BC0183E05C
:104B80008093CB06CE010E949F23B0C081E080932A
:104B9000CB068FA584FF03C060E070E003C0B801BE
:104BA0006F5F7F4FCE0144E08CC0843039F4E091D8
:104BB000D406F091D506309789F432C0833099F548
:104BC00084E08093CB06E091D406F091D50630972F
:104BD00039F18EA582958F70482F50E0440F551FF4
:104BE000440F551FC70108974E5D5F4F8417950707
:104BF00008F4AC01C801840F951FE816F90610F0FF
:104C0000980103C09701241B350B8DA182958695D1
:104C1000877060E00995882319F0CE01B8010BC0B8
:104C2000CE01B8014DC0853009F460C030FF0AC024
:104C30006F5F7F4FCE0149E00E94C72385E08093DC
:104C4000CB0654C00115110509F452C0CE0138C07D
:104C50008091D106981709F049C09DA180918705E0
:104C6000981709F043C08FA581FF04C0CE010E94B0
:104C700017243CC084FF3AC0988980E02989422FDC
:104C800050E0482B592B2EA5822F82958F7090E0F3
:104C9000880F991F880F991F481B590B445150408A
:104CA00057FF02C040E050E05093D3064093D20635
:104CB000452B51F48FA580FF19C0CE0160E070E054
:104CC00040E00E94C72312C08EA582958F70682F86
:104CD00070E0660F771F660F771F6E5D7F4F88EF5E
:104CE0009FEFE80EF91EE616F70610F460E070E09C
:104CF000CB01DF91CF911F910F91FF90EF9008951D
:104D000082E080938305F2CF8FA5382F82FDECCE11
:104D1000FDCE0895CB01BA010E943A1F0895CB0140
:104D2000BA010E94B62408952F923F925F926F922B
:104D30007F928F929F92AF92BF92CF92DF92EF922B
:104D4000FF920F931F93DF93CF93CDB7DEB72A97D0
:104D50000FB6F894DEBF0FBECDBF3B015A83498327
:104D60003C832B83FE82ED82D886CF82BA86A986C9
:104D700014010E948828AC01CB01DA014C015D01CD
:104D8000C3016B817C814D815E812F8138850985CE
:104D90001A857101CE8CDF8C0E949A1D88E0582EF6
:104DA00089819A81B3010E943A1F8C01C301B80125
:104DB0000E94B624892BA1F7C301B8010E94601D8F
:104DC0000E94361B853011F481E026C00E9488289D
:104DD000A50194012059384E4F4F5F4F26173707D2
:104DE00048075907E8F60E9488285A94A1F0AC01B8
:104DF000CB01DA014C015D01C3016B817C814D81E6
:104E00005E812F81388509851A857101CE8CDF8CF2
:104E10000E949A1DC5CF80E02A960FB6F894DEBF97
:104E20000FBECDBFCF91DF911F910F91FF90EF90FB
:104E3000DF90CF90BF90AF909F908F907F906F90BA
:104E40005F903F902F900895CB010E945C220895BF
:104E5000CB01BA010E94FE230895CB01BA01A9013A
:104E60000E9470220895CB01BA01A9010E94F42189
:104E70000895CB01BA01A9010E943C210895CF9366
:104E8000DF93CB01642F0E94082082E00E94F61E6F
:104E90006AE070E080E090E00E949628C0E0D0E0F8
:104EA00084E160E878E30E94EA1F64EF71E080E04B
:104EB00090E00E94962884E160E979E30E94EA1F6D
:104EC00064EF71E080E090E00E9496282196C33064
:104ED000D10531F784E166E774E30E94EA1F64E6D6
:104EE00070E080E090E00E949628DF91CF910895D5
:104EF0004AE00E943F2708950E94221E0895F999D2
:104F0000FECF72BD61BDF89A80B50895F999FECFC4
:104F10001FBA72BD61BD40BD0FB6F894FA9AF99AF6
:104F20000FBE08958091F7069091F806089560935A
:104F3000890570938A0580938B0590938C0508955D
:104F40006093EF067093F0068093F1069093F2065B
:104F50002091890530918A0540918B0550918C05EF
:104F6000260F371F481F591F2093F3063093F4066E
:104F70004093F5065093F60682E090E09093F80691
:104F80008093F7060E9488286093F9067093FA06CA
:104F90008093FB069093FC060895EF92FF920F9387
:104FA0001F931CC02F5F3F4F4F4F5F4F2093EF0663
:104FB0003093F0064093F1065093F20688EE93E0AA
:104FC000A0E0B0E0E80EF91E0A1F1B1FE092F906F0
:104FD000F092FA060093FB061093FC060E948828C4
:104FE000E090F906F090FA060091FB061091FC069D
:104FF0006E197F09800B910B2091EF063091F0061E
:105000004091F1065091F206685E734080409040F6
:1050100048F68091F3069091F406A091F506B091C0
:10502000F606281739074A075B07E8F0E091ED0616
:10503000F091EE06309749F00995611571058105EB
:10504000910519F00E94A0270EC020E030E0809169
:10505000F7069091F806892B11F021E030E03093AB
:10506000F8062093F7066091EF067091F0068091A4
:10507000F1069091F2061F910F91FF90EF90089525
:105080001F920F920FB60F9211242F933F938F937D
:105090009F93AF93BF938091010790910207A091D6
:1050A0000307B0910407309105070196A11DB11DBA
:1050B000232F2D5F2D3720F02D570196A11DB11DF7
:1050C000209305078093010790930207A09303079D
:1050D000B09304078091FD069091FE06A091FF0613
:1050E000B09100070196A11DB11D8093FD0690931C
:1050F000FE06A093FF06B0930007BF91AF919F916A
:105100008F913F912F910F900FBE0F901F90189588
:105110008FB7F8942091010730910207409103075F
:10512000509104078FBFB901CA0108959B01AC01DA
:105130007FB7F8948091FD069091FE06A091FF063E
:10514000B091000766B5A89B05C06F3F19F00196A6
:10515000A11DB11D7FBFBA2FA92F982F8827860FB9
:10516000911DA11DB11D62E0880F991FAA1FBB1FD1
:105170006A95D1F7BC012DC0FFB7F8948091FD0668
:105180009091FE06A091FF06B0910007E6B5A89B9E
:1051900005C0EF3F19F00196A11DB11DFFBFBA2F49
:1051A000A92F982F88278E0F911DA11DB11DE2E018
:1051B000880F991FAA1FBB1FEA95D1F7861B970B73
:1051C000885E9340C8F221503040404050406851C2
:1051D0007C4F211531054105510571F60895019760
:1051E00039F0880F991F880F991F02970197F1F7DF
:1051F0000895789484B5826084BD84B5816084BD4F
:1052000085B5826085BD85B5816085BDEEE6F0E03F
:10521000808181608083E1E8F0E01082808182609B
:105220008083808181608083E0E8F0E0808181601C
:105230008083E1EBF0E0808184608083E0EBF0E04C
:10524000808181608083EAE7F0E0808184608083F0
:10525000808182608083808181608083808180689A
:1052600080831092C1000895982F8E3008F09E50D0
:10527000977080918D058295880F880F807C892B8F
:1052800080937C0080917A00806480937A00809182
:105290007A0086FDFCCF2091780040917900942F10
:1052A00080E030E0282B392BC9010895CF93DF939C
:1052B000482F50E0CA0183589B4FFC013491475955
:1052C0005B4FFA018491882369F190E0880F991F60
:1052D000FC01E55BFB4FA591B491FC01EB5AFB4F40
:1052E000C591D491662351F42FB7F8948C91932FE4
:1052F000909589238C93888189230BC0623061F457
:105300002FB7F8948C91932F909589238C93888153
:10531000832B88832FBF06C09FB7F8948C91832B73
:105320008C939FBFDF91CF910895482F50E0CA0121
:105330008F569B4FFC012491CA0183589B4FFC015F
:10534000949147595B4FFA013491332309F440C0DB
:10535000222351F1233071F0243028F42130A1F0C0
:10536000223011F514C02630B1F02730C1F02430BE
:10537000D9F404C0809180008F7703C080918000B1
:105380008F7D8093800010C084B58F7702C084B574
:105390008F7D84BD09C08091B0008F7703C080915C
:1053A000B0008F7D8093B000E32FF0E0EE0FFF1F81
:1053B000EB5AFB4FA591B4912FB7F894662321F4D3
:1053C0008C919095892302C08C91892B8C932FBF4F
:1053D0000895682F70E0CB018F569B4FFC012491FC
:1053E000CB0183589B4FFC01449167597B4FFB01D4
:1053F0009491992319F420E030E03CC0222351F12C
:10540000233071F0243028F42130A1F0223011F53E
:1054100014C02630B1F02730C1F02430D9F404C0D4
:10542000809180008F7703C0809180008F7D809372
:10543000800010C084B58F7702C084B58F7D84BD95
:1054400009C08091B0008F7703C08091B0008F7D3C
:105450008093B000892F90E0880F991F815A9B4F4D
:10546000FC01A591B4918C9120E030E0842311F0EF
:1054700021E030E0C901089508951F920F920FB600
:105480000F9211242F933F934F938F939F93EF93FA
:10549000FF938091C00082FD1DC04091C600209105
:1054A0004607309147072F5F3F4F2F733070809131
:1054B0004807909149072817390771F0E09146078E
:1054C000F0914707EA5FF84F4083309347072093F6
:1054D000460702C08091C600FF91EF919F918F9186
:1054E0004F913F912F910F900FBE0F901F901895E5
:1054F000E0919A07F0919B07E05CFF4F81919191B9
:1055000020813181821B930B8F739070892B11F056
:105510000E943C2A08951F920F920FB60F921124F9
:105520002F933F938F939F93EF93FF9320918A073D
:1055300030918B0780918C0790918D072817390740
:1055400031F48091C1008F7D8093C10014C0E0913F
:105550008C07F0918D07E65BF84F208180918C07D6
:1055600090918D0701968F73907090938D07809323
:105570008C072093C600FF91EF919F918F913F91EF
:105580002F910F900FBE0F901F901895AF92BF9262
:10559000DF92EF92FF920F931F93CF93DF93EC0173
:1055A0007A018B01DD24403081EE580780E06807E6
:1055B00080E0780711F0DD24D39491E0A92EB12C7E
:1055C000EC89FD89DD2069F0C50108A002C0880FC3
:1055D000991F0A94E2F7808360E079E08DE390E020
:1055E00005C0108260E874E88EE190E0A8019701A0
:1055F0000E943D2E215030404040504056954795E6
:105600003795279580E12030380720F0DD2011F014
:10561000DD24D6CFE889F9893083EA89FB892083A4
:1056200019A2EE89FF89408121E030E0C9010C8C8C
:1056300002C0880F991F0A94E2F7482B4083EE8935
:10564000FF894081C9010D8C02C0880F991F0A94FF
:10565000E2F7482B4083EE89FF894081C9010E8C17
:1056600002C0880F991F0A94E2F7482B4083EE8905
:10567000FF8980810F8C02C0220F331F0A94E2F74A
:10568000209528232083DF91CF911F910F91FF90C8
:10569000EF90DF90BF90AF900895DC011C96ED91E4
:1056A000FC911D97E05CFF4F2191319180819181A8
:1056B000281B390B2F733070C9010895DC011C962B
:1056C000ED91FC911D97E05CFF4F20813181E0540A
:1056D000F040DF01AE5BBF4F8D919C911197281771
:1056E000390719F42FEF3FEF07C08D919C91E80F18
:1056F000F91F8081282F30E0C9010895DC011C9634
:10570000ED91FC911D97E05CFF4F20813181E054C9
:10571000F040DF01AE5BBF4F8D919C911197281730
:10572000390719F42FEF3FEF10C08D919C9111971D
:10573000E80FF91F20818D919C91119701968F732D
:10574000907011969C938E9330E0C9010895DC010E
:1057500091968C919197882339F05496ED91FC9114
:105760005597808186FFF9CF91961C920895CF932B
:10577000DF93EC01EE85FF85E05CFF4F20813181F6
:10578000E054F0402F5F3F4F2F733070DF01AE5B6E
:10579000BF4F8D919C91119728173907D1F3E05C89
:1057A000FF4F80819181E054F040E80FF91F608342
:1057B000EE85FF85E05CFF4F31832083EE89FF8912
:1057C000208181E090E00F8C02C0880F991F0A941D
:1057D000E2F7282B208381E089A3EC89FD89808171
:1057E0008064808381E090E0DF91CF91089581E033
:1057F0000895109291071092900788EE93E0A0E030
:10580000B0E08093920790939307A0939407B0938E
:10581000950782E995E090938F0780938E0786E045
:1058200097E090939B0780939A078AE497E0909380
:105830009D0780939C0785EC90E090939F07809351
:105840009E0784EC90E09093A1078093A00780ECE2
:1058500090E09093A3078093A20781EC90E090934F
:10586000A5078093A40782EC90E09093A70780930C
:10587000A60786EC90E09093A9078093A80784E0A0
:105880008093AA0783E08093AB0787E08093AC07FF
:1058900085E08093AD0781E08093AE070895CF93B4
:1058A000DF930E94F9280E94CA19C8E7DAE20E9431
:1058B00069172097E1F30E94782AF9CFCF92DF92FF
:1058C000EF92FF920F931F93CF93DF937C016B01B5
:1058D0008A01C0E0D0E00FC0D6016D916D01D70103
:1058E000ED91FC910190F081E02DC7010995C80F61
:1058F000D91F015010400115110571F7CE01DF913C
:10590000CF911F910F91FF90EF90DF90CF9008956E
:10591000DC01ED91FC910190F081E02D0995089555
:10592000EF92FF920F931F938C01DC01ED91FC919C
:105930000190F081E02D6DE009957C01D801ED9199
:10594000FC910190F081E02DC8016AE009959C016D
:105950002E0D3F1DC9011F910F91FF90EF900895EB
:10596000CF93DF93EC016115710519F420E030E06D
:105970000FC0DB010D900020E9F71197A61BB70BB4
:10598000E881F9810280F381E02DAD0109959C0148
:10599000C901DF91CF9108954F925F927F928F92CC
:1059A0009F92AF92BF92CF92DF92EF92FF920F93AE
:1059B0001F93DF93CF93CDB7DEB7A1970FB6F894BF
:1059C000DEBF0FBECDBF2C01742ECB01223008F4F8
:1059D0002AE019A231E2C32ED12CCC0EDD1E822E7C
:1059E0009924AA24BB24672D752FA50194010E9438
:1059F0003D2E79018A01C801B701A50194010E94D9
:105A0000F72D472D461B0894C108D1084A3014F4DD
:105A1000405D01C0495CF6014083E114F1040105D9
:105A2000110521F07E2C5F2DC801DDCFC201B6012A
:105A30000E94B02CA1960FB6F894DEBF0FBECDBF6A
:105A4000CF91DF911F910F91FF90EF90DF90CF905A
:105A5000BF90AF909F908F907F905F904F900895F0
:105A6000DC012115310541F4ED91FC910190F081AB
:105A7000E02D642F099508950E94CC2C0895EF9293
:105A8000FF920F931F939A01E62EFF2400E010E08F
:105A9000B801A7010E94302D1F910F91FF90EF9048
:105AA0000895CF92DF92EF92FF920F931F93CF93BF
:105AB000DF93EC016A017B012115310541F4E88196
:105AC000F9810190F081E02D642F09951FC02A30E3
:105AD0003105D1F477FF17C0E881F9810190F08199
:105AE000E02D6DE209958C0144275527BA014C1928
:105AF0005D096E097F09CE012AE00E94CC2C980135
:105B0000280F391F04C02AE00E94CC2C9C01C90137
:105B1000DF91CF911F910F91FF90EF90DF90CF9089
:105B20000895EF92FF920F931F937B019A01002734
:105B3000F7FC0095102FB801A7010E94512D1F916D
:105B40000F91FF90EF9008950E94B02C0895CF938D
:105B5000DF93EC010E948828688779878A879B8772
:105B6000E881F9810680F781E02DCE0109959C013D
:105B700097FF15C00E948828288539854A855B854E
:105B8000621B730B840B950B2C813D814E815F81D1
:105B9000621773078407950718F32FEF3FEFC901CA
:105BA000DF91CF910895CF92DF92EF92FF920F9302
:105BB0001F93CF93DF936C018B017A01C0E0D0E09B
:105BC00009C0C6010E94A72D97FD07C0F801819367
:105BD0008F012196CE15DF05A0F3CE01DF91CF9185
:105BE0001F910F91FF90EF90DF90CF900895629FEB
:105BF000D001739FF001829FE00DF11D649FE00DC5
:105C0000F11D929FF00D839FF00D749FF00D659F25
:105C1000F00D9927729FB00DE11DF91F639FB00D24
:105C2000E11DF91FBD01CF0111240895AA1BBB1B63
:105C300051E107C0AA1FBB1FA617B70710F0A61B8C
:105C4000B70B881F991F5A95A9F780959095BC01AD
:105C5000CD01089597FB092E07260AD077FD04D0C1
:105C6000E5DF06D000201AF4709561957F4F089506
:105C7000F6F7909581959F4F0895A1E21A2EAA1BE1
:105C8000BB1BFD010DC0AA1FBB1FEE1FFF1FA217EC
:105C9000B307E407F50720F0A21BB30BE40BF50BE9
:105CA000661F771F881F991F1A9469F76095709572
:105CB000809590959B01AC01BD01CF01089597FBA4
:105CC000092E05260ED057FD04D0D7DF0AD0001CC0
:105CD00038F450954095309521953F4F4F4F5F4F89
:105CE0000895F6F790958095709561957F4F8F4F49
:105CF0009F4F0895EE0FFF1F0590F491E02D09943A
:105D00002F923F924F925F926F927F928F929F92CB
:105D1000AF92BF92CF92DF92EF92FF920F931F93B9
:105D2000CF93DF93CDB7DEB7CA1BDB0B0FB6F8946A
:105D3000DEBF0FBECDBF09942A88398848885F84AA
:105D40006E847D848C849B84AA84B984C884DF801B
:105D5000EE80FD800C811B81AA81B981CE0FD11DFF
:105D60000FB6F894DEBF0FBECDBFED010895F894D5
:025D7000FFCF63
:105D72003F50313D002650323D002650333D002633
:105D820050343D002650323D310047455420002F0B
:105D920020002E0001000000545556212223C0A8E5
:105DA2000119C0A80101C0A80101C0A80101FFFF9B
:105DB200FF00501A4F9033C83240003A00204E0084
:105DC2000010270000020000000000000000000098
:105DD20000000000000000000000000000000000C1
:105DE20000000000000000000000000000000000B1
:105DF20000000000000000000000000000000000A1
:105E02000000000000000000000000000000000090
:1061E2000000000000000041726475696E6F2D307E
:1061F20030000A01010001500A2C010000010000D8
:0E6202000000B72B5E2C4D2B7E2B5E2BA72BA6
:00000001FF
